:100000000C946B000C9493000C9493000C9493004C
:100010000C9493000C94DA050C9493000C949300C8
:100020000C9493000C9493000C9493000C94930004
:100030000C9493000C9493000C9493000C949300F4
:100040000C946A100C9493000C949B030C9475030D
:100050000C9493000C9493000C9493000C949300D4
:100060000C94CD030C949300B402C302D2021D037E
:10007000E102F002FF020E0300000000240027004E
:100080002A0000000000250028002B0000000000CE
:1000900023002600290004040404040404040202CA
:1000A00002020202030303030303010204081020F7
:1000B0004080010204081020010204081020000002
:1000C0000008000201000003040700000000000017
:1000D00000002C15B41011241FBECFEFD4E0DEBFFA
:1000E000CDBF23E0A4E0B2E001C01D92AE3FB20755
:1000F000E1F712E0A0E0B1E0E2E1F4E302C0059034
:100100000D92A430B107D9F710E0CAE6D0E004C0E0
:100110002197FE010E949616C936D107C9F70E94A1
:10012000C0100C94FC190C940000CF92DF92EF9257
:10013000FF920F931F93CF93DF936C017A018B0192
:10014000C0E0D0E0CE15DF0581F0D8016D918D01C2
:10015000D601ED91FC910190F081E02DC601099549
:10016000892B11F02196EECF7E01C701DF91CF914F
:100170001F910F91FF90EF90DF90CF900895FC01B9
:10018000538D448D252F30E0842F90E0821B930BFC
:10019000541710F0CF96089501970895FC01918DA2
:1001A000828D981761F0828DDF01A80FB11D5D96D9
:1001B0008C91928D9F5F9F73928F90E008958FEF47
:1001C0009FEF0895FC01918D828D981731F0828DFB
:1001D000E80FF11D858D90E008958FEF9FEF089552
:1001E000FC01918D228D892F90E0805C9F4F821BB6
:1001F00091098F73992708958FED92E00E94F00086
:1002000021E0892B09F420E0822F0895FC01848DE0
:10021000DF01A80FB11DA35ABF4F2C91848D90E030
:1002200001968F739927848FA689B7892C93A0890B
:10023000B1898C91837080648C93938D848D981395
:1002400006C00288F389E02D80818F7D8083089528
:10025000EF92FF920F931F93CF93DF93EC0181E016
:10026000888F9B8D8C8D981305C0E889F9898081D2
:1002700085FD26C0F62E0B8D10E00F5F1F4F0F730C
:100280001127E02E8C8DE8120CC00FB607FCFACFB8
:10029000E889F989808185FFF5CFCE010E940601AA
:1002A000F1CF8B8DFE01E80FF11DE35AFF4FF08275
:1002B0009FB7F8940B8FEA89FB89808180620AC01E
:1002C0009FB7F894EE89FF896083E889F989808176
:1002D0008370806480839FBF81E090E0DF91CF9145
:1002E0001F910F91FF90EF900895CF93DF93EC0152
:1002F000888D8823C9F0EA89FB89808185FD05C046
:10030000A889B9898C9186FD0FC00FB607FCF5CF7F
:10031000808185FFF2CFA889B9898C9185FFEDCFC7
:10032000CE010E940601E7CFDF91CF91089580E0D2
:1003300090E0892B29F00E94FC0081110C940000B0
:10034000089585ED8093BC008091BC0084FDFCCFB6
:100350001092B902089540913402262F30E0240F04
:10036000311D21323105DCF42091B9022430C9F469
:10037000FC0180E090E0861758F43091340221911E
:10038000DC01AC5EBD4FA30FB11D2C930196F3CFE2
:1003900080913402680F6093340280E0089581E018
:1003A000089582E00895089508950895E0917202F5
:1003B00080917102E81730F4F0E0ED58FD4F808134
:1003C00090E008958FEF9FEF0895909172028091D1
:1003D0007102981750F4E92FF0E0ED58FD4F20819D
:1003E00030E09F5F9093720202C02FEF3FEFC90190
:1003F00008958091710290E020917202821B910910
:100400000895CF92DF92EF92FF920F931F93CF93B5
:10041000DF937C01CB018A012091BA02222389F06B
:10042000EB016B01C40ED51ECC15DD0569F0699199
:10043000D701ED91FC910190F081E02DC701099564
:10044000F3CF642F0E94AB01C801DF91CF911F91C0
:100450000F91FF90EF90DF90CF900895CF93DF93AF
:100460001F92CDB7DEB769832091BA022223D1F063
:100470002091DD02203240F021E030E0FC013383A6
:10048000228380E090E015C08091BB02E82FF0E06D
:10049000E454FD4F998190838F5F8093BB028093DA
:1004A000DD0205C061E0CE0101960E94AB0181E052
:1004B00090E00F90DF91CF910895089580E090E053
:1004C0000895CF93DF93EC0160E08E810E94B90F15
:1004D00061E08E810E94B90F60E08E810E94B90FA9
:1004E0008BE891E00197F1F7DF91CF910895CF92DA
:1004F000DF92EF92FF920F931F93CF93DF93EB0165
:100500007B0124E0E20EF11C8B016C01C61AD70AB4
:10051000C601800F911F0E94FD15F80181938F0184
:10052000EE15FF05A9F7CE01DF91CF911F910F9135
:10053000FF90EF90DF90CF9008950E94E71961E05F
:1005400083E00E940D0E84E691E00E94700EE0911F
:10055000DE028E2F90E08830910508F06EC0FC011D
:10056000EC5CFF4F0C94961680E492E4AFE0B0E0B0
:1005700080930E0190930F01A0931001B09311018D
:100580008AE691E068C080EA96E8A1E0B0E0809356
:100590000E0190930F01A0931001B093110183E716
:1005A00091E059C080E197E2A0E0B0E080930E01B5
:1005B00090930F01A0931001B09311018CE791E08B
:1005C0004AC084E690E0A0E0B0E080930E019093F2
:1005D0000F01A0931001B09311018EE891E03BC090
:1005E0008AE090E0A0E0B0E080930E0190930F01CC
:1005F000A0931001B093110187E991E02CC081E034
:1006000090E0A0E0B0E080930E0190930F01A093E2
:100610001001B093110180EA91E01DC08AE090E0E2
:10062000A0E0B0E080930E0190930F01A093100121
:10063000B093110189EA91E00EC088EE93E0A0E04A
:10064000B0E080930E0190930F01A0931001B0933E
:10065000110185E891E00E94690F61E088E00E9445
:100660000D0E0E944C0F0C94720EEF92FF920F939E
:100670001F93CF93DF93EC017B018A0188819981DD
:10068000009729F02A813B8124173507F8F4B80137
:100690006F5F7F4F0E942119009759F099838883DB
:1006A0001B830A832C813D81232B81F4FC01108262
:1006B0000DC088819981009711F00E9498181982C5
:1006C00018821D821C821B821A8207C01D830C8324
:1006D000B701888199810E94F519CE01DF91CF91F0
:1006E0001F910F91FF90EF9008951F920F920FB6F8
:1006F0000F9211242F933F934F935F936F937F93A8
:100700008F939F93AF93BF93EF93FF938FED92E0FF
:100710000E940601FF91EF91BF91AF919F918F9140
:100720007F916F915F914F913F912F910F900FBEED
:100730000F901F9018951F920F920FB60F921124D1
:100740002F938F939F93EF93FF93E091EF02F0919C
:10075000F0028081E091F502F091F60282FD12C074
:1007600090818091F8028F5F8F732091F902821738
:1007700051F0E091F802F0E0E152FD4F958F809347
:10078000F80201C08081FF91EF919F918F912F918D
:100790000F900FBE0F901F9018951F920F920FB6DB
:1007A0000F9211242F933F934F935F936F937F93F7
:1007B0008F939F93AF93BF93EF93FF938091B90073
:1007C000887F803609F49CC068F5883209F45BC0E4
:1007D00090F4803109F454C038F4882309F4F6C049
:1007E000883009F44DC0F6C0883109F44CC080321D
:1007F00009F45DC0EFC0803409F468C048F4803368
:1008000009F455C0883309F0E5C08093B702D8C019
:10081000803509F44FC0883509F45DC0883409F08B
:10082000D9C0D6C0883909F4C7C0A8F4883709F4FC
:1008300067C038F4883609F463C0803709F460C0B3
:10084000C9C0883809F4B8C0803909F45FC080385D
:1008500009F0C0C05BC0803B09F486C038F4803A20
:1008600009F466C0883A09F47FC0B4C0803C09F43A
:10087000A7C0883C09F4A4C0883B09F48AC0AAC078
:100880008091940210C09091B6028091B5029817A1
:1008900070F5E091B60281E08E0F8093B602F0E031
:1008A000EB56FD4F80818093BB0085EC86C0809322
:1008B000B7028EC0E091B60281E08E0F8093B6023F
:1008C0008091BB00F0E0EB56FD4F80839091B60223
:1008D0008091B5026EC0E091B60281E08E0F8093E8
:1008E000B6028091BB00F0E0EB56FD4F8083809113
:1008F000B80281116DC081E08093930284EA61C0E7
:1009000083E08093B90210925602CFCF80915602B5
:10091000803208F051C0E091560281E08E0F809342
:1009200056028091BB00F0E0EA5CFD4F8083BDCFB2
:1009300085EC8093BC001092B902809156028032FF
:1009400030F4E0915602F0E0EA5CFD4F10826091D5
:10095000560270E0E0916D02F0916E0286E392E043
:1009600009951092560236C084E08093B902109225
:10097000350210923402E0916F02F09170020995F5
:1009800080913402811105C081E08093340210927D
:100990001402E091350281E08E0F80933502F0E081
:1009A000EC5EFD4F80818093BB0090913502809179
:1009B0003402981708F479CF85E88093BC000AC008
:1009C00085EC8093BC001092B90204C01092B7026B
:1009D0000E94A101FF91EF91BF91AF919F918F91E3
:1009E0007F916F915F914F913F912F910F900FBE2B
:1009F0000F901F901895CF92DF92EF92FF920F9376
:100A00001F93CF93DF936C017C0187E0E80EF11C0C
:100A1000C0E0D0E0062F10E0B8010C2E02C07595A2
:100A200067950A94E2F76170F70181917F010E9456
:100A3000B90F2196C430D10579F7C601DF91CF9166
:100A40001F910F91FF90EF90DF90CF900C94610277
:100A5000CF92DF92EF92FF920F931F93CF93DF938A
:100A6000EC01F62E642F8C810E94B90F8D818F3F8F
:100A700019F060E00E94B90F8F850F2D10E084FF00
:100A800025C06E0187E0C80ED11CE12CF12CB80105
:100A90000E2C02C0759567950A94E2F76170F60115
:100AA00081916F010E94B90FFFEFEF1AFF0A88E0F2
:100AB000E816F10461F7CE01DF91CF911F910F91FC
:100AC000FF90EF90DF90CF900C946102B80184E02A
:100AD000759567958A95E1F7CE010E94FB046F2D0D
:100AE000CE01DF91CF911F910F91FF90EF90DF909A
:100AF000CF900C94FB0441E00E94280581E090E037
:100B00000895FF920F931F93CF93DF93EC01F62E7E
:100B100008811981C8010E94FD15F81621F06F2D7A
:100B2000C8010E940516CE01DF91CF911F910F9150
:100B3000FF900895AF92BF92CF92DF92EF92FF9213
:100B40000F931F93CF93DF9300D0CDB7DEB78B0108
:100B50006B0124E0C20ED11C7B015C01A61AB70A0E
:100B6000C5018E0D9F1DF70161917F019A838983D5
:100B7000CE0101960E948105EC14FD0489F7C8019D
:100B80000F900F90DF91CF911F910F91FF90EF90F9
:100B9000DF90CF90BF90AF9008956AE071E080E061
:100BA00090E00E949A0581E090E090930501809387
:100BB000040108951F920F920FB60F921124CF9245
:100BC000DF92EF92FF922F933F934F935F936F9338
:100BD0007F938F939F93AF93BF93CF93DF93EF93C5
:100BE000FF938091F0030E94900FEC018091EF033E
:100BF0000E94900FE091EE03EF70CC0FDD1F8C2B65
:100C000034E0E39FF0011124E85EFE4FE80FF11D90
:100C1000C081C093EE03C07309F470C10E945E10DE
:100C2000C0905702D0905802E0905902F0905A02BA
:100C30009B01AC012C193D094E095F092093670205
:100C4000309368024093690250936A02609357029E
:100C5000709358028093590290935A0280916B02CC
:100C600090916C02C03109F06EC0892B09F044C02C
:100C700040910A0150910B0160910C0170910D019E
:100C800080910E0190910F01A0911001B09111017E
:100C9000840F951FA61FB71F80930A0190930B0125
:100CA000A0930C01B0930D0160910A0170910B01AA
:100CB00080910C0190910D0120910E0130910F0156
:100CC0004091100150911101C0900E01D0900F0180
:100CD000E0901001F09011010E947416C701B60156
:100CE0000E94641660930A0170930B0180930C01BB
:100CF00090930D010E94CD0580916B0290916C0242
:100D0000019709F0AEC060E071E084E190E00E94DC
:100D1000770240910E0150910F0160911001709186
:100D20001101FC0180819181A281B381840F951F03
:100D3000A61FB71F8093000190930101A0930201A9
:100D4000B093030188C0892B09F044C080910A0147
:100D500090910B01A0910C01B0910D0140910E01F9
:100D600050910F016091100170911101841B950B3E
:100D7000A60BB70B80930A0190930B01A0930C0173
:100D8000B0930D0160910A0170910B0180910C01EB
:100D900090910D0120910E0130910F0140911001B1
:100DA00050911101C0900E01D0900F01E090100100
:100DB000F09011010E947416C701B6010E946416DA
:100DC00060930A0170930B0180930C0190930D01C5
:100DD0000E94CD0580916B0290916C02019709F001
:100DE00040C060E071E084E190E00E9477024091B1
:100DF0000E0150910F016091100170911101FC01E1
:100E000080819181A281B381841B950BA60BB70BC6
:100E10008093000190930101A0930201B09303011C
:100E200060E071E084E190E00E949A058091000109
:100E300090910101A0910201B091030118161906C9
:100E40001A061B0674F01092000110920101109214
:100E500002011092030160E071E084E190E00E94E1
:100E60009A0580910A0190910B01A0910C01B0911B
:100E70000D018130914EA54FB54080F08091060163
:100E800090910701A0910801B091090180930A0196
:100E900090930B01A0930C01B0930D0180910A0176
:100EA00090910B01A0910C01B0910D01803A9648F0
:100EB000A140B10580F48091060190910701A091B5
:100EC0000801B091090180930A0190930B01A0934E
:100ED0000C01B0930D0160E071E084E190E00E94AC
:100EE0007702FC0180819181A281B381809300010E
:100EF00090930101A0930201B0930301FF91EF9140
:100F0000DF91CF91BF91AF919F918F917F916F9121
:100F10005F914F913F912F91FF90EF90DF90CF9095
:100F20000F900FBE0F901F9018950F931F93CF93A4
:100F3000DF938B0191E09093BA0290E69093DC02EC
:100F40001092BB021092DD02682F8CE793E00E94A2
:100F50002E02E801085F1F4F69918CE793E00E9421
:100F60002E02C017D107C1F781E0DF91CF911F9109
:100F70000F910C94880ECF93DF9391E09093BA0277
:100F800090E69093DC021092BB021092DD02682F73
:100F90008CE793E00E942E0281E00E94880E8091EF
:100FA000B9028111FCCF81E08093B9021092B8029E
:100FB0009FEF9093B7021092B6021092B502809301
:100FC000940280919402806C8093940280919302A9
:100FD000813061F410929302809194028093BB005F
:100FE0008091BC0083FDF8CF85EC01C085EE809335
:100FF000BC008091B9028130E1F38091B602811189
:1010000003C0C091B60201C0C1E0E5E9F2E0A3E788
:10101000B2E080E08C1721F091919D938F5FFACF21
:1010200010927202C093710280917202C81731F05F
:101030008CE793E00E94E501D82FF6CF8D2FDF914A
:10104000CF9108952F923F924F925F926F927F922D
:101050008F929F92AF92BF92CF92DF92EF92FF92C8
:101060000F931F93CF93DF93CDB7DEB761970FB682
:10107000F894DEBF0FBECDBF2D833E834F835887CC
:1010800069877A871C011F870E876091EA03709138
:10109000EB038091EC039091ED0324E630E040E017
:1010A00050E00E94F5162D87388B4B875C87762E93
:1010B000672E582E492E8091E4039091E503A0916C
:1010C000E603B091E7036C017D01FF0CCC08DC2C3A
:1010D00076019C01AD016C2D7C2D8C2D9C2D0FE19A
:1010E0000E94C017A12C0AECB02EEAE9CE2EFBE339
:1010F000DF2EE12CF12C00E010E00E942217AD84DD
:10110000B888CB84DC84E72CF62C052D142D0E94A6
:101110009C160FE10E94DB1749015A01D501C40159
:10112000BB0F880B982FDC0189839A83AB83BC8328
:101130009401A5016981762F862F962FAD84B888FA
:10114000CB84DC84E72CF62C052D0E94F71729832D
:10115000832E942E598B688B7B878C879D872D815E
:101160003E814F81588569857A85C1012F3FA7E56A
:101170003A07A7E44A07A8EF5A07ADE06A077105E6
:1011800081059105A9F0A0F0211534404B46544F3C
:101190006441710581059105B9F0B0F01D8294E0BC
:1011A0009E83ABE6AF83B4EFB887E4E1E98709C07B
:1011B0001D82E8E5EE83F7E4FF8328EF28878DE0C2
:1011C00089871A86212C312CA980B82CC92CD98862
:1011D000E888FB840C851D852D813E814F815885D3
:1011E00069857A85C1010E94531729013A01FFE000
:1011F0004F1651046104710418F4AFE0AA2E08C020
:101200002BE54216510461047104D0F0FAE5AF2ECB
:10121000B12CC12CD12CE12CF12C00E010E0298163
:10122000382D492D598968897B858C859D850E943B
:101230009C162D833E834F83588769877A871C01CC
:10124000A980B82CC92CD988E888FB840C851D8519
:101250002D813E814F81588569857A85C1010E9423
:101260005117AA24AA94BB24BA94EFE0CE2ED12C15
:10127000E12CF12C00E010E00E949C16A980B82C13
:10128000C92CD988E888FB840C851D850E945317DA
:10129000C901DA010097A105B10529F4C12CD12CAF
:1012A0007601C39406C0CC24CA94DC2C5FE0E52E02
:1012B000F12CBC01CD0127E0660F771F881F991F15
:1012C0002A95D1F737E0440C551C661C771C3A95DB
:1012D000D1F7A2E05A1A61087108A70196010E948D
:1012E0007416862E372E982E420E531E641E751EBF
:1012F00084E190E00E9400189A838983FC01D082E7
:10130000C182862D8370828353824482D701C601B5
:101310004CE0B695A795979587954A95D1F7807F2C
:10132000C82EC90CC582368287828E859F85892BFF
:1013300019F4BF018AE107C0AE85BF85119729F472
:1013400069817A8182E20E94950789819A816196FA
:101350000FB6F894DEBF0FBECDBFDF91CF911F91C6
:101360000F91FF90EF90DF90CF90BF90AF909F9044
:101370008F907F906F905F904F903F902F900C9444
:10138000981810927202109271021092BB02109281
:10139000DD021092B90281E08093B80210929302AC
:1013A00061E082E10E94B90F61E083E10E94B90F20
:1013B000E9EBF0E080818E7F808380818D7F808368
:1013C00088E48093B80085E48093BC0083ED91E0CD
:1013D0009093700280936F0284ED91E090936E027F
:1013E00080936D0208950E94C10962E987EB0E9413
:1013F000E40E8FE00E94BB0740EC5CEF6BE971E00C
:101400004093EA035093EB036093EC037093ED0376
:10141000682F6F738FE00E94E40E60E880E10E9405
:10142000E40E60E881E10E94E40E60E882E10E943F
:10143000E40E6CE080E10E94E40E6CE081E10E9429
:10144000E40E6CE082E10E94E40E60E281EB0E9417
:10145000E40E60E881EB0C94E40E2F923F924F92E1
:101460005F926F927F928F929F92AF92BF92CF9234
:10147000DF92EF92FF920F931F93CF93DF93CDB73D
:10148000DEB761970FB6F894DEBF0FBECDBF8901FE
:10149000772E898B9F872F3FE4E33E07ECE04E07D2
:1014A00051056105710581059105B1F1A8F1422E43
:1014B000312E642E552E262E2115304A4C4A594B7A
:1014C000634071058105910569F060F0412CB0EA37
:1014D0003B2E1CEA612E09EB502E83E0282E712C46
:1014E000198A1F86242D332D462D552D622D772DDB
:1014F00089899F8535534C405109610971098109DA
:1015000091092F3F34434C40510561057105810518
:10151000910509F000F50AC0412CF5E33F2EACE03F
:101520006A2E512C212C712C198A1F86242D332DC3
:10153000462D552D622D772D89899F8507E00E94C4
:10154000C017422E332E642E552E262E772E898BD1
:101550009F87B7E014C1242D332D462D552D622DC4
:10156000772D89899F853A5648415109610971094A
:10157000810991092F3F394648415105610571059F
:101580008105910509F0A8F4242D332D462D552D04
:10159000622D772D89899F8506E00E94C017422E13
:1015A000332E642E552E262E772E898B9F87F6E0BC
:1015B000B7C0242D332D462D552D622D772D8989C9
:1015C0009F85345D40435109610971098109910981
:1015D0002F3F334D4043510561057105810591054C
:1015E00009F0A8F4242D332D462D552D622D772D8D
:1015F00089899F8505E00E94C017422E332E642EF4
:10160000552E262E772E898B9F87B5E0B8C0242DC6
:10161000332D462D552D622D772D89899F85385A7A
:101620004146510961097109810991092F3F374AE2
:1016300041465105610571058105910509F0A8F440
:10164000242D332D462D552D622D772D89899F858B
:1016500004E00E94C017422E332E642E552E262EF3
:10166000772E898B9F87F4E05BC0242D332D462D88
:10167000552D622D772D89899F853055434C510911
:1016800061097109810991092F3F3F44434C51057C
:10169000610571058105910509F0A8F4242D332D0C
:1016A000462D552D622D772D89899F8503E00E9457
:1016B000C017422E332E642E552E262E772E898B60
:1016C0009F87B3E05CC0242D332D462D552D622D10
:1016D000772D89899F85305A4648514061097109A3
:1016E000810991092F3F3F494648514061057105E5
:1016F0008105910509F0B0F4242D332D462D552D8B
:10170000622D772D89899F8502E00E94C017422EA5
:10171000332E642E552E262E772E898B9F87F2E04E
:10172000FD8343C0242D332D462D552D622D772D5D
:1017300089899F8530544D40534061097109810961
:1017400091092F3F3F434D4053406105710581058D
:10175000910509F0B0F4242D332D462D552D622D21
:10176000772D89899F8501E00E94C017422E332E74
:10177000642E552E262E772E898B9F87B1E0BD8350
:1017800014C0242D332D462D552D622D772D89899A
:101790009F852F3F354D41415E476340710581056F
:1017A000910511F008F0B3C01D82A42CB32CC62CF7
:1017B000D52CE22CF72C09891F8520E03CE343E57A
:1017C0005CE460E170E080E090E00E9453172983C0
:1017D0003A834B835C8389819A81AB81BC81069774
:1017E000A105B10570F49AEA9E83A4E3AF83B3E642
:1017F000B887E7EBE987F2E0FA87912C812C1B860A
:1018000009C04E823F82688659862A86972C89882D
:101810002F852B87AE80BF80C884D984EA84F92CB9
:10182000082D1B8520E03CE343E55CE460E170E0CB
:1018300080E090E00E945117AA24AA94BB24BA9495
:10184000EFE0CE2ED12CE12CF12C00E010E00E9434
:101850009C16AE80BF80C884D984EA84F92C082DF8
:101860001B850E945317C901DA010097A105B10534
:1018700029F4C12CD12C7601C39406C0CC24CA947F
:10188000DC2C6FE0E62EF12CBC01CD0147E0660FA9
:10189000771F881F991F4A95D1F789809A80AB805E
:1018A000BC8057E0880C991CAA1CBB1C5A95D1F728
:1018B000A2E09A1AA108B108A70196010E94741625
:1018C000820E931EA41EB51E6D877E87082F409240
:1018D000C9033092CA036092CB035092CC0320928A
:1018E000CD037092CE03B989B093CF03EF85E09317
:1018F000D00310E01982FCE3FE8323E52F838CE400
:10190000888790E199871A861B861C8651C0242DF2
:10191000332D462D552D622D772D89899F8502E027
:101920000E94C01729833E834F83588769877A872F
:101930008B879C8780E10E94BB07682F6F7D80E1C9
:101940000E94E40EA981A093B903BE81B093BA03AB
:10195000EF81E093BB03F885F093BC0329852093C6
:10196000BD038A858093BE039B859093BF03AC859E
:10197000A093C0034092C9033092CA036092CB0384
:101980005092CC032092CD037092CE03B989B093CC
:10199000CF03EF85E093D003C12CD12C7601C39403
:1019A0001D861E8600E0812C912C54011D8211E0C1
:1019B00084E190E00E940018988B8F87DC01DC9214
:1019C0001196CC928CE20E94BB079A2D93708C7F6B
:1019D000892BEF85F889828393828482D701C6019F
:1019E0002CE0B695A795979587952A95D1F7807F96
:1019F000C82EC00EC5822E8526838D858783BF01A4
:101A00008AE20E94950780E10E94BB07682F11308F
:101A100011F4606401C06F7B80E10E94E40E1093BA
:101A2000E1038CE20E94BB07837811118C60AD81C9
:101A300090E1A99FB0011124682B8CE20E94E40E72
:101A40008F8598890E949818113061F400E010E0A9
:101A500029813E814F81588569857A858B859C8552
:101A60000E94220880E061960FB6F894DEBF0FBE98
:101A7000CDBFDF91CF911F910F91FF90EF90DF903D
:101A8000CF90BF90AF909F908F907F906F905F901E
:101A90004F903F902F900895009769F0FC010190BE
:101AA0000020E9F73197AF01481B590BBC0188E9C9
:101AB00093E00C94950080E090E0089540E0682F5A
:101AC00088E993E00C94280581E00E945E0D8BE389
:101AD0009FE10197F1F70895CF93DF93823028F0CB
:101AE0009091A70398609093A7038093AB03109203
:101AF000AC0380E48093AD0380E18093AE0380E586
:101B00008093AF0361E080919C030E94E80F809175
:101B10009D038F3F19F061E00E94E80F61E0809122
:101B20009E030E94E80FC8E9D3E09E012859334084
:101B30008091A70384FD03C084E090E002C088E0A8
:101B400090E02196281739072CF461E08E810E94DD
:101B5000E80FEBCF8BE39DE00197F1F760E0809118
:101B60009C030E94B90F60E080919E030E94B90F10
:101B700080919D038F3F19F060E00E94B90F809122
:101B8000A70384FD20C063E088E993E00E94FB0482
:101B9000CBE4D6E4CE010197F1F763E088E993E066
:101BA0000E94FB042197F1F763E088E993E00E942B
:101BB000FB0483E592E00197F1F762E088E993E0A6
:101BC0000E94FB0415C080620E945E0D8BE496E4C7
:101BD0000197F1F78091A70380620E945E0D83E573
:101BE00092E00197F1F78091A70380620E945E0D59
:101BF0008091A70380620E945E0D84E08093A80319
:101C00008CE00E945E0D0E94640D82E08093A90327
:101C100086E0DF91CF910C945E0D643008F063E0B4
:101C20009091AB03691710F06FEF690FE62FF0E0AA
:101C3000E856FC4F9489890F80680C945E0D41E052
:101C4000682F88E993E00E94280581E090E00895DC
:101C50008F929F92AF92BF920F931F93CF93DF9378
:101C6000CDB7DEB7A1970FB6F894DEBF0FBECDBFDC
:101C700019A2423008F44AE08E010F5D1F4F842EF6
:101C8000912CA12CB12CA50194010E947416E62F71
:101C9000B901CA0101501109EA3014F4E05D01C034
:101CA000E95CD801EC93232B242B252B61F7C80189
:101CB0000E944C0DA1960FB6F894DEBF0FBECDBFAB
:101CC000DF91CF911F910F91BF90AF909F908F9018
:101CD0000895682F70E080E090E04AE00C94280EB0
:101CE0000C944C0DCF93DF9300D0CDB7DEB760914D
:101CF000DE028EE190E09A838983CE0101960E94F4
:101D000081058EED92E00F900F90DF91CF910895B5
:101D1000282F3091DD02313208F04AC08091B9029B
:101D20008111FCCF9091DC0242E04093B9022093F4
:101D3000B8022FEF2093B7021092B6023093B5028B
:101D4000ECEBF2E0A5E9B2E020E0321721F041919E
:101D50004D932F5FFACF1092940220919402990F25
:101D6000922B9093940290919302913061F410928F
:101D70009302909194029093BB009091BC0093FDCC
:101D8000F8CF95EC01C095EE9093BC009091B9020C
:101D90009230E1F39091B7029F3F79F08091B702C2
:101DA000803241F08091B702803331F084E005C089
:101DB00081E003C082E001C083E01092BB02109278
:101DC000DD021092BA020895CF93C62F91E090934E
:101DD000BA0290E69093DC021092BB021092DD02F0
:101DE000682F8CE793E00E942E026C2F8CE793E023
:101DF0000E942E0281E0CF910C94880E833081F0F6
:101E000028F4813099F08230A1F008958730A9F04C
:101E10008830B9F08430D1F4809180008F7D03C088
:101E2000809180008F7780938000089584B58F77AC
:101E300002C084B58F7D84BD08958091B0008F77F6
:101E400003C08091B0008F7D8093B00008953FB7AC
:101E5000F8948091F6039091F703A091F803B09164
:101E6000F90326B5A89B05C02F3F19F00196A11DC7
:101E7000B11D3FBFBA2FA92F982F8827820F911D20
:101E8000A11DB11DBC01CD0142E0660F771F881F67
:101E9000991F4A95D1F70895E2E9F3E0448155810D
:101EA0006081718188E993E00C94950080E48093CF
:101EB0007C0080917A00806480937A0080917A001F
:101EC00086FDFCCF809178002091790090E0922BE4
:101ED0000895009771F0FC0101900020E9F7319717
:101EE000AF01481B590BBC0182E993E00E94350306
:101EF00014C08091920390919303009711F00E9477
:101F000098181092930310929203109297031092D4
:101F10009603109295031092940382E993E008953A
:101F2000CF93DF93282F30E0F901E254FF4F8491E3
:101F3000F901E655FF4FD491F901EA56FF4FC491DC
:101F4000CC2391F081110E94FE0EEC2FF0E0EE0FF9
:101F5000FF1FE457FF4FA591B491EC91ED2381E071
:101F600090E021F480E002C080E090E0DF91CF912A
:101F700008951F93CF93DF93282F30E0F901E254A7
:101F8000FF4F8491F901E655FF4FD491F901EA56CC
:101F9000FF4FC491CC23C1F0162F81110E94FE0E79
:101FA000EC2FF0E0EE0FFF1FEE57FF4FA591B4911D
:101FB0009FB7F894111104C08C91D095D82302C01A
:101FC000EC91DE2BDC939FBFDF91CF911F910895A1
:101FD000CF93DF9390E0FC01E655FF4F2491FC0185
:101FE000EA56FF4F8491882361F190E0880F991F92
:101FF000FC01E858FF4FC591D491FC01EE57FF4F0B
:10200000A591B491611109C09FB7F894888120957A
:1020100082238883EC912E230BC0623061F49FB73A
:10202000F8948881322F309583238883EC912E2B6E
:102030002C939FBF06C08FB7F894E8812E2B28837E
:102040008FBFDF91CF9108958F929F92AF92BF92F1
:10205000CF92DF92EF92FF926B017C010E94270FDB
:102060004B015C01C114D104E104F104F1F00E94C0
:10207000270FDC01CB0188199909AA09BB09883E01
:102080009340A105B10570F321E0C21AD108E1081F
:10209000F10888EE880E83E0981EA11CB11CC114C3
:1020A000D104E104F10419F7DDCFFF90EF90DF9048
:1020B000CF90BF90AF909F908F9008952FB7F894D6
:1020C0006091F2037091F3038091F4039091F50312
:1020D0002FBF08951F920F920FB60F9211242F93C6
:1020E0003F938F939F93AF93BF938091F20390910F
:1020F000F303A091F403B091F5033091F10323E0D1
:10210000230F2D3720F40196A11DB11D05C026E82F
:10211000230F0296A11DB11D2093F1038093F203BA
:102120009093F303A093F403B093F5038091F60327
:102130009091F703A091F803B091F9030196A11DC6
:10214000B11D8093F6039093F703A093F803B09327
:10215000F903BF91AF919F918F913F912F910F9074
:102160000FBE0F901F90189580918C0390918D0356
:102170000E94981880919203909193030C94981860
:10218000CF93DF9300D0CDB7DEB7789484B582606B
:1021900084BD84B5816084BD85B5826085BD85B50B
:1021A000816085BD80916E00816080936E00109289
:1021B0008100809181008260809381008091810004
:1021C0008160809381008091800081608093800095
:1021D0008091B10084608093B1008091B0008160F3
:1021E0008093B00080917A00846080937A0080911F
:1021F0007A00826080937A0080917A008160809377
:102200007A0080917A00806880937A001092C100F1
:10221000E091EF02F091F00282E08083E091EF0222
:10222000F091F0021082E091EB02F091EC0210824A
:10223000E091ED02F091EE0280E180831092F702CE
:10224000E091F302F091F40286E08083E091F102E4
:10225000F091F202808180618083E091F102F0913F
:10226000F202808188608083E091F102F091F202B5
:10227000808180688083E091F102F091F202808198
:102280008F7D808382E00E946C0D0E94640D0E940D
:10229000C10960E08EE00E94E80F61E08EE00E94DC
:1022A000B90F8091680084608093680080916D0010
:1022B0008C6080936D0078940E94640D60E080E0F3
:1022C0000E940D0E82EB91E00E94700E61E080E0B2
:1022D0000E940D0E83EC91E00E94700E68EC70E09D
:1022E00080E090E00E94241061E080E00E940D0EEA
:1022F00068E572E080E090E00E94241000E110E0C8
:1023000088E10E945E0D62E370E080E090E00E9450
:10231000241001501109A1F70E94640D8AE090E099
:102320000E94FD1580935B028A3F09F074C30E94EE
:10233000560F853F914034F00E94560F8C3B9240DF
:102340000CF469C36AE071E080E090E00E947702DB
:102350008EE190E00E94FD158093DE0261E083E053
:102360000E940D0E84E691E00E94700E61E088E00C
:102370000E940D0E0E944C0F0E945E106093570247
:10238000709358028093590290935A0284E690E029
:10239000A0E0B0E08093670290936802A093690286
:1023A000B0936A020E94F30900E010E020E03CE3F1
:1023B00043E55CE460E170E080E090E00E94220888
:1023C00060910A0170910B0180910C0190910D01B7
:1023D00024E630E040E050E00E94F5160E942D0A0D
:1023E00060E071E084E190E00E947702FC0180816E
:1023F0009181A281B3818093000190930101A09308
:102400000201B09303018093E4039093E503A0934A
:10241000E603B093E7030E94F30920E03CE343E5C1
:102420005CE460E170E080E090E00E94220883E0DC
:102430000E94BB07682F6E7F83E00E94E40E83E05A
:102440000E94BB07682F626083E00E94E40E83E075
:102450000E94BB07682F646083E00E94E40E80E165
:102460000E94BB07682F636080E10E94E40E8AE04F
:10247000C82ED12CE12CF12C98EE492E93E0592E48
:10248000612C712C22242394312C80916B02909129
:102490006C02892B09F0D6C060910A0170910B0182
:1024A00080910C0190910D0120E432E44FE050E066
:1024B0000E947416B22E122F2093620260910A01BC
:1024C00070910B0180910C0190910D0120EA36E88A
:1024D00041E050E00E947416CA01B901A7019601BB
:1024E0000E9474166093610260910A0170910B0161
:1024F00080910C0190910D0120E137E240E050E025
:102500000E947416CA01B901A70196010E947416AF
:102510006093600260910A0170910B0180910C013F
:1025200090910D01A30192010E947416CA01B90194
:10253000A70196010E94741660935F0260910A01E0
:1025400070910B0180910C0190910D0124E630E017
:1025500040E050E00E947416CA01B901A70196013B
:102560000E94741660935E0260910A0170910B01E3
:1025700080910C0190910D01A70196010E947416A3
:10258000CA01B901A70196010E94741660935D0209
:1025900060910A0170910B0180910C0190910D01E5
:1025A000A70196010E94741660935C0260E080E0CF
:1025B0000E940D0E80E20E941F0E80E20E941F0EFC
:1025C00060E01A3010F081E001C082E00E940D0E40
:1025D0008B2D0E94690E84ED91E00E94700E809117
:1025E00061020E94690E809160020E94690E8091D2
:1025F0005F020E94690E84ED91E00E94700E80914E
:102600005E020E94690E80915D020E94690E8091B7
:102610005C020E94690E8EE691E00E94700E80E2DC
:102620000E941F0E0E945E106093880370938903BE
:1026300080938A0390938B031092050110920401FA
:102640000E949F020E94560F0E94560F5C019093B9
:102650006602809365026AE070E080E090E00E948C
:1026600024100E94560F0E94560F092E000CAA0B30
:10267000BB0BA5010B2C000C660B770B8C019D018D
:1026800003501109210931094017510762077307E7
:1026900064F00396A11DB11D84179507A607B7071F
:1026A00024F0B0926402A092630280916302909140
:1026B00064028351924087379105A0F560E080E085
:1026C0000E940D0E86ED91E00E94700E61E081E0A7
:1026D0000E940D0E81E092E00E94700E8090000139
:1026E00090900101A0900201B0900301B7FE0CC0D0
:1026F0008DE20E941F0E66277727CB0168197909A2
:102700008A099B094AE003C04AE0C501B4010E945E
:10271000280E87EF91E00E94700E30926C0220929A
:102720006B0204C010926C0210926B028091DE0268
:10273000873009F0ADC08091670290916802A09146
:102740006902B0916A028D329140A105B105C0F0D5
:10275000C0920E01D0920F01E0921001F09211018F
:1027600040926702509268026092690270926A0217
:1027700061E080E00E940D0E80E092E00E94700E09
:102780008091670290916802A0916902B0916A02FB
:102790008C549109A109B109813E9105A105B105AA
:1027A00000F584E690E0A0E0B0E080930E01909305
:1027B0000F01A0931001B09311018BEB90E0A0E00A
:1027C000B0E08093670290936802A0936902B0938F
:1027D0006A0261E080E00E940D0E88EE91E00E94A6
:1027E000700E8091670290916802A0916902B09189
:1027F0006A024A97A109B109C297A105B105E0F49F
:1028000040920E0150920F016092100170921101DE
:1028100082E390E0A0E0B0E08093670290936802CA
:10282000A0936902B0936A0261E080E00E940D0EFD
:102830008CEE91E00E94700E809167029091680288
:10284000A0916902B0916A024A97A105B10500F50D
:1028500088EA91E6A0E0B0E080930E0190930F012A
:10286000A0931001B093110184E190E0A0E0B0E0EA
:102870008093670290936802A0936902B0936A0202
:1028800061E080E00E940D0E80EF91E00E94700EEA
:1028900040910A0150910B0160910C0170910D0162
:1028A0008091060190910701A0910801B091090162
:1028B000481759076A077B0709F45AC080910A0133
:1028C00090910B01A0910C01B0910D018130914EBE
:1028D000A54FB54080F08091060190910701A0912D
:1028E0000801B091090180930A0190930B01A09314
:1028F0000C01B0930D0180910A0190910B01A09100
:102900000C01B0910D01803A9648A140B10580F4C8
:102910008091060190910701A0910801B0910901F1
:1029200080930A0190930B01A0930C01B0930D01C9
:1029300060910A0170910B0180910C0190910D0141
:1029400024E630E040E050E00E94F5160E942D0A97
:1029500080910A0190910B01A0910C01B0910D01A1
:102960008093060190930701A0930801B093090199
:102970008091040190910501892BE9F40E945E1079
:10298000009188031091890320918A0330918B0371
:1029900004521A4F2F4F3F4F60177107820793075A
:1029A00050F00E94CD0540926702509268026092FA
:1029B000690270926A028EE00E94900F892B41F5A5
:1029C0008091DE028F5F883018F48093DE0202C0AF
:1029D0001092DE020E949F0268EC70E080E090E0BE
:1029E0000E94241061E080E00E940D0E8DEE91E0C7
:1029F0000E94700E68EC70E080E090E00E9424106D
:102A000061E080E00E940D0E81E092E00E94700E75
:102A10000E9497013ACD60E071E084E190E00E946D
:102A20009A058AE090E09A8389836AEFCE01019645
:102A30000E9481058BE090E09A83898360E0CE015B
:102A400001960E9481056AE071E080E090E00E94BA
:102A50009A050E94720E76CCCF93DF93EFEDF2E0F1
:102A60001382128288EE93E0A0E0B0E08483958325
:102A7000A683B78328E331E03183208325EC30E05F
:102A80003587248724EC30E03787268720EC30E038
:102A9000318B208B21EC30E0338B228B22EC30E029
:102AA000358B248B26EC30E0378B268B118E128EE3
:102AB000138E148EECE7F3E01382128284839583E5
:102AC000A683B7838AE491E091838083CEEED3E03E
:102AD00083E0898382E08A8360E083E00E94E80FDC
:102AE00060E08A810E94E80F61E089810E94B90F4D
:102AF00061E08A810E94B90F1882E0EBF3E088E080
:102B000080AF81AF11AA12AA13AA1186128613866A
:102B10001486158616861786108A118A128A138AD9
:102B2000148A158A168A178A108E118E128E138EA9
:102B3000148E158E168E178E10A211A212A213A239
:102B400014A215A216A217A210A611A612A613A6C9
:102B500014A615A616A617A610AA40EC5CEF6BE902
:102B600071E042AF53AF64AF75AFE8E9F3E01382B1
:102B700012822CE531E03183208399E094839FEF2A
:102B80009583868387E0878386E0808785E08187D9
:102B900084E082871386148615861686178681E060
:102BA0000E946C0DE2E9F3E011821082138212821E
:102BB000158214824FE050E064EF71E0CF010E9473
:102BC0003503ECE8F3E01182108213821282158241
:102BD000148240E050E063E072E0CF010E943503D0
:102BE0000E945E10609388037093890380938A0328
:102BF00090938B03DF91CF910895F999FECF92BD09
:102C000081BDF89A992780B50895262FF999FECFAE
:102C10001FBA92BD81BD20BD0FB6F894FA9AF99AF9
:102C20000FBE019608950E945516A59F900DB49F62
:102C3000900DA49F800D911D112408952F923F9215
:102C40004F925F926F927F928F929F92AF92BF92BC
:102C5000CF92DF92EF92FF920F931F93CF93DF9368
:102C6000CDB7DEB7CA1BDB0B0FB6F894DEBF0FBEC5
:102C7000CDBF09942A88398848885F846E847D8412
:102C80008C849B84AA84B984C884DF80EE80FD8014
:102C90000C811B81AA81B981CE0FD11D0FB6F8948A
:102CA000DEBF0FBECDBFED010895A29FB001B39F5F
:102CB000C001A39F700D811D1124911DB29F700D45
:102CC000811D1124911D0895DB018F939F930E9414
:102CD0001316BF91AF91A29F800D911DA39F900DE0
:102CE000B29F900D11240895A1E21A2EAA1BBB1BBE
:102CF000FD010DC0AA1FBB1FEE1FFF1FA217B307C8
:102D0000E407F50720F0A21BB30BE40BF50B661FDD
:102D1000771F881F991F1A9469F7609570958095A1
:102D200090959B01AC01BD01CF010895EE0FFF1FEF
:102D30000590F491E02D0994DF93CF931F930F93A7
:102D40009A9DF02D219FF00D8B9DF00D8A9DE02D19
:102D5000F10D039FF00D029FE00DF11D4E9DE00D62
:102D6000F11D5E9DF00D4F9DF00D7F936F93BF920F
:102D7000AF925F934F93D5010E9455168B01AC0122
:102D8000D7010E945516EB01E80FF91FD6010E94EA
:102D9000EC162F913F91D6010E945516C60FD71FF2
:102DA000E81FF91FAF91BF910E94EC162F913F9140
:102DB0000E945516C60FD71FE81FF91FD6010E94A3
:102DC0005516E60FF71F9801BE01CF0111240F9190
:102DD0001F91CF91DF9108950E945516460F571FFE
:102DE000C81FD91F08F431960895E894DF93CF9354
:102DF000FC01DB010E9455167F936F93E9019A0154
:102E0000AC01BF93AF933F932F93DF010E94551600
:102E100026F46C1B7D0B820B930B9E01EB01FC01D6
:102E20000E94EC16AF91BF912F913F910E94EC163A
:102E3000BE01CF01F9012F913F91CF91DF9108950C
:102E4000689401C0E894F92FF12B12F00C945417F8
:102E5000A0E0B0E0EEE2F7E10C942416092E059410
:102E600022F40E94B017112392F4F0E80F26FFEF2E
:102E7000E094F09400951095B094C094D094A194EF
:102E8000BF0ACF0ADF0AEF0AFF0A0F0B1F0B0E94CF
:102E90005F1707FC0E94B017CDB7DEB7ECE00C94CB
:102EA0004016689401C0E8948F929F92CF93DF936D
:102EB0000E945F17DF91CF919F908F900895882493
:102EC0009924F401E401B0E49F93AA279A158B0496
:102ED0009C04ED05FE05CF05D007A10798F4AD2FA2
:102EE000DC2FCF2FFE2FE92D982C892E982F872F9E
:102EF000762F652F542F432F322F2227B85031F7CA
:102F0000BF9127C01B2EBF91BB27220F331F441F29
:102F1000551F661F771F881F991F881C991CEE1F5D
:102F2000FF1FCC1FDD1FAA1FBB1F8A149B04EC05CB
:102F3000FD05CE05DF05A007B10748F08A189B08FC
:102F4000EC09FD09CE09DF09A00BB10B21601A9431
:102F5000E1F62EF49401AF01BE01CD01000C0895FD
:102F600060957095809590953095409550952195F8
:102F70003F4F4F4F5F4F6F4F7F4F8F4F9F4F089582
:102F80000F93083090F0982F872F762F652F542FAE
:102F9000432F322F22270850F4CF220F331F441F14
:102FA000551F661F771F881F991F0A95B2F70F914B
:102FB000089597FB10F8169400080F93083098F0C6
:102FC0000850232F342F452F562F672F782F892F06
:102FD000902DF4CF0594979587957795679557959C
:102FE0004795379527950A95AAF70F9108952A0DC9
:102FF0003B1D4C1D5D1D6E1D7F1D801F911F089583
:103000000F931F93CF93DF938230910510F482E0EA
:1030100090E0E091FC03F091FD0320E030E0A0E0BF
:10302000B0E0309719F14081518102811381481736
:103030005907C8F08417950769F4109731F0129674
:103040000C93129713961C9327C00093FC031093C4
:10305000FD0322C02115310519F04217530718F45A
:103060009A01BD01EF01DF01F801DBCF2115310528
:10307000F9F0281B390B2430310580F48A819B81BB
:103080006115710521F0FB019383828304C0909345
:10309000FD038093FC03FE01329644C0FE01E20F63
:1030A000F31F8193919322503109398328833AC0C9
:1030B0002091FA033091FB03232B41F4209114015A
:1030C000309115013093FB032093FA0320911201F4
:1030D000309113012115310541F42DB73EB74091D0
:1030E000160150911701241B350BE091FA03F09162
:1030F000FB03E217F307A0F42E1B3F0B2817390739
:1031000078F0AC014E5F5F4F2417350748F04E0F43
:103110005F1F5093FB034093FA038193919302C086
:10312000E0E0F0E0CF01DF91CF911F910F91089582
:10313000CF93DF93009709F481C0FC01329713828B
:103140001282A091FC03B091FD03109781F42081BD
:103150003181820F931F2091FA033091FB032817CE
:10316000390751F5F093FB03E093FA0367C0ED01D3
:1031700020E030E0CE17DF0740F44A815B819E01FA
:1031800041155105F1F0EA01F5CFD383C2834081A7
:103190005181840F951FC817D90759F488819981E7
:1031A000840F951F0296918380838A819B819383EC
:1031B00082832115310529F4F093FD03E093FC038C
:1031C0003DC0E901FB83EA8349915991C40FD51FA2
:1031D000EC17FD0761F480819181840F951F0296A1
:1031E000E90199838883828193819B838A83E0E0CC
:1031F000F0E012968D919C911397009719F0FD01C4
:10320000DC01F7CF8D919C9111979D012E5F3F4F6F
:10321000820F931F2091FA033091FB03281739077F
:1032200069F4309729F41092FD031092FC0302C058
:1032300013821282B093FB03A093FA03DF91CF9124
:103240000895A0E0B0E0E7E2F9E10C942216EC0169
:10325000009721F4CB010E940018B4C0FC01E60FD6
:10326000F71F9C0122503109E217F30708F4A8C0A8
:10327000D9010D911C91119706171707B0F0053071
:10328000110508F49BC0C80104978617970708F436
:1032900095C002501109061B170B019311936D93F2
:1032A0007C93CF010E94981889C05B01A01AB10AD3
:1032B0004C01800E911EA091FC03B091FD03612C86
:1032C000712CE12CF12C109709F446C08D919C9142
:1032D0001197A815B905B1F56C0142E0C40ED11CD7
:1032E000CA14DB0478F14C018A189B08640142E09F
:1032F000C40ED11C1296BC9012971396AC91B5E0F7
:10330000CB16D10440F0B282A38391828082D9018E
:103310006D937C9309C00E5F1F4F800F911FF901C1
:1033200091838083EB2DFA2FE114F10431F0D70162
:103330001396FC93EE93129741C0F093FD03E09334
:10334000FC033CC06816790608F43C017D01129626
:103350000D90BC91A02DB7CF8091FA039091FB0303
:1033600088169906E1F466167706C8F48091120172
:1033700090911301009741F48DB79EB740911601CB
:1033800050911701841B950BE817F907C8F4F093C7
:10339000FB03E093FA03F901718360830FC0CB0153
:1033A0000E9400187C01009759F0A801BE010E94FC
:1033B000EC19CE010E949818C70104C0CE0102C0CA
:1033C00080E090E0CDB7DEB7EEE00C943E1681E0F1
:1033D00090E0F8940C94FC19FB01DC0102C0019010
:1033E0000D9241505040D8F70895FB01DC01019047
:1033F0000D920020E1F7089510E0CAE6D0E004C085
:10340000FE010E9496162196CB36D107C9F7F89493
:02341000FFCFEC
:10341200D847030001000100000080969800A086B2
:1034220001000000FE0380000002040003000110FE
:10343200030200000302010006000400060500204A
:10344200060504000000000028019500BF00750178
:10345200F000CE00E200000000002E0201025E0237
:10346200D501F901E501D601000000007B059500B8
:103472005E025D02537465703A0020202031204DB7
:10348200487A0020313030204B487A0020203130F9
:10349200204B487A0020202031204B487A002020FF
:1034A20031303020487A00202020313020487A0004
:1034B200202020312020487A0020202020417574CD
:1034C2006F0053693533353120204175746F737441
:1034D2006570003130304B487A2E2E2E2E3130302E
:1034E2004D487A002E00436F72722E504C4C20537E
:1034F20069353335312020003E2020003E3E200039
:103502003E3E3E002020202020202020202020207F
:043512002020200055
:00000001FF
